:020000040000FA
:06000000B4EF26F012002F
:060008003DEF26F012009E
:0600180044EF26F0120087
:06080000B4EF26F0120027
:06082A000200AC4D0000CD
:10083000E000000011000000AA4D0000AF01000020
:0408400002000000B2
:0C0844000F0E8A1693161200C1EC0CF087
:10085000060E0001FB5D05E36D50020B01E0120086
:1008600001D81200D9CFE6FFE1CFD9FF3B0EE12638
:100870003C0EE66E410EE66E070EE66EE3EC21F0EE
:10088000E552E552E5520701006FE850000802E327
:10089000D6EF0AF044C716F044C717F0166A435162
:1008A00000011610146E44C715F0390E14C0DBFF9A
:1008B0003A0E44C7DBFF070141513A0A02E1FAEF61
:1008C00008F0010A02E1FAEF08F0070A02E1FAEF84
:1008D00008F0040A01E1F8D3780A01E1EBD37F0ABA
:1008E00001E13AD3010A01E1D5D1070A01E19BD127
:1008F0000D0A01E17AD1020A01E169D1010A01E19F
:10090000FAD0020A01E1DFD0060A71E0010A02E032
:10091000B2EF0AF0530E016F42C702F7390EDBCF78
:1009200014F03A0EDBCF15F0800E145CFF0E155854
:1009300033E3390EDBCF14F03A0EDBCF15F0800E27
:10094000145EFF0E155A010E14C0DBFF020EDB6AA7
:100950004251F36E020EDBCFF4FFF350F45C02E37E
:10096000C5EF0AF0010EDBCFF3FFDB2AF350EA6A92
:10097000600FE96E000EEA22EF50E66E020EDB50C9
:10098000040FEA6A010FE96E070EEA22E552E7500A
:10099000EF6E020EDB2ADCD7020EDB6A0701425142
:1009A000F36E020EDBCFF4FFF350F45C02E3C5EF0D
:1009B0000AF0390EDBCFE6FF3A0EDBCFE6FF48EC5C
:1009C00019F0E552E552E66E020EDB50040FEA6ABA
:1009D000010FE96E070EEA22E552E750EF6E020EB4
:1009E000DB2A390EDB2A3A0ED9E3DB2AD7D7520E9F
:1009F000016F42C702F7390EDBCF14F03A0EDBCF9E
:100A000015F0800E145CFF0E155836E3390EDBCF5F
:100A100014F03A0EDBCF15F0800E145EFF0E155A5F
:100A20007F0E1416000E1516010E14C0DBFF020E09
:100A3000DB6A4251F36E020EDBCFF4FFF350F45C3D
:100A400002E3C5EF0AF0020EDB50040FEA6A410F21
:100A5000E96E070EEA22EF50E66E010EDB50EA6AFD
:100A6000600FE96E000EEA22E552E750EF6E020ECB
:100A7000DB2A010EDB2ADDD7390EDBCFE6FF3A0E8B
:100A8000DBCFE6FFC80E146E3B0E156E166A14C05F
:100A9000E6FFE66E16C0E6FFD950050FE66E000EC3
:100AA000DA20E66E2BEC24F0F56E070EE15EF550D1
:100AB000D950050FE66E000EDA20E66E63EC13F0F7
:100AC000E552E552ABD08B70520E016F42C702F770
:100AD000390EDBCFE6FF3A0EDBCFE6FF94EC18F0E1
:100AE000E552E552E76E020EE7CFDBFFDB5002E195
:100AF000C5EF0AF093D0520E016F42C702F7390ECC
:100B0000DBCF14F03A0EDBCF15F0800E145CFF0E35
:100B1000155835E3390EDBCF14F03A0EDBCF15F064
:100B2000800E145EFF0E155A7F0E1416000E151659
:100B3000010E14C0DBFF020EF36EDB6E4251F36E4A
:100B4000020EDBCFF4FFF350F45C1BE2020EDB502D
:100B5000040FEA6A410FE96E070EEA22EF50E66ED3
:100B6000010EDB50EA6A600FE96E000EEA22E552E0
:100B7000E750EF6E020EDB2A010EDB2ADFD7510EA3
:100B8000016F8B7046C716F046C717F0166A07014B
:100B9000455100011610146E46C715F0390E14C0E9
:100BA000DBFF3A0E46C7DBFF390EDBCFE6FF3A0E1E
:100BB000DBCFE6FF94EC18F0E552E552E76E020E4B
:100BC000E7CFDBFFDB5002E1C5EF0AF027D0520E82
:100BD000016F42C702F7390EDBCFE6FF3A0EDBCFDB
:100BE000E6FF33EC18F0C3EF0AF0520E016F42C774
:100BF00002F7D950390FE96EDACFEAFFEE50ED1067
:100C000003E08990C5EF0AF08CEC19F0E76E010E55
:100C1000E7CFDBFFDB5002E1C5EF0AF00701510E21
:100C2000016FC5EF0AF0520E016F42C702F7B90E0D
:100C3000146E3B0E156E166A14C0E6FFE66E16C003
:100C4000E6FF33EC13F0E552E552E552B3EC1BF04E
:100C5000020EDB6A500EF36E020EDBCFF4FFF35090
:100C6000F45C02E3C5EF0AF0020EDB50EA6A520FB1
:100C7000E96E010EEA22EF50E66E020EDB50EA6AE0
:100C8000600FE96E000EEA22E552E750EF6E020EA9
:100C9000DB2AE0D7520E016F42C702F79E0E146E98
:100CA0003B0E156E166A14C0E6FFE66E16C0E6FF30
:100CB00033EC13F0E552E552E5526DEC1BF0A00E5B
:100CC000E66E7BEC1BF0E552010EDB6A030EDB6A7D
:100CD000040EDB6A010EDB50146E156AD8901550B5
:100CE00004E6CF0E145C000E155801E37ED0070E0B
:100CF000E76E030EDBCFF6FF040EDBCFF7FFE75006
:100D0000F616F76A8F0EF626470EF7220800F51C36
:100D1000146E030EDBCFE9FF040EDBCFEAFF030EF8
:100D2000D890EA32E932E804FBE1020EE926010E2E
:100D3000EA221450EF16030EDB2A040E01E3DB2A2D
:100D4000070EE76E030EDBCFF6FF040EDBCFF7FFD7
:100D5000E750F616F76A8F0EF626470EF7220800C0
:100D6000F51C146E030EDBCFE9FF040EDBCFEAFFA8
:100D7000030ED890EA32E932E804FBE1020EE926DC
:100D8000010EEA221450EF16030EDB2A040E01E3D3
:100D9000DB2A070EE76E030EDBCFF6FF040EDBCF78
:100DA000F7FFE750F616F76A8F0EF626470EF72282
:100DB0000800F5CF14F0030EDBCFE9FF040EDBCF04
:100DC000EAFF030ED890EA32E932E804FBE1020EB2
:100DD000E926010EEA221450EF12030EDB2A040E5C
:100DE00001E3DB2A010EDB2A75D70101400E006FFB
:100DF000040EE66EECEC1AF0E5528A92010EDB6A04
:100E0000500EF36E010EDBCFF4FFF350F45C0BE2F7
:100E1000010EDB50EA6A520FE96E010EEA22EF6A18
:100E2000010EDB2AEDD7030EDB6A040EDB6A030E2C
:100E3000DBCF14F0040EDBCF15F0D890155004E68C
:100E40006C0E145C020E15586BE28B92030EE66E6C
:100E5000C0EC26F0E552070EE76E030EDBCFF6FF7F
:100E6000040EDBCFF7FFE750F616F76A8F0EF62673
:100E7000470EF7220800F5CF14F0030EDBCFE9FF91
:100E8000040EDBCFEAFF030ED890EA32E932E80421
:100E9000FBE1020EE926010EEA22EF50141402E0F3
:100EA000010E01D0000E010BF36EFE0E8A14F3103A
:100EB0008A6E030EE66EC0EC26F0E55282A424D0C2
:100EC000070EE76E030EDBCFF6FF040EDBCFF7FF56
:100ED000E750F616F76A8F0EF626470EF72208003F
:100EE000F5CF14F0030EDBCFE9FF040EDBCFEAFFF2
:100EF000030ED890EA32E932E804FBE1520EE9260B
:100F0000010EEA221450EF128B82030EE66EC0EC43
:100F100026F0E552030EDB2A040E89E3DB2A87D78D
:100F20008A828B92930EF66E470EF76E0800F5508C
:100F300001014F1502E0010E01D0000E010BF36E0E
:100F4000FE0E8A14F3108A6E030EE66EC0EC26F0D5
:100F5000E55282A496D08DD0520E016F42C702F79F
:100F6000650E146E3B0E156E166A14C0E6FFE66E33
:100F700016C0E6FF33EC13F0E552E552E5526DEC96
:100F80001BF0A00EE66E7BEC1BF0E5520101400E5B
:100F9000006F040EE66EECEC1AF0E5528A92010E38
:100FA000DB6A500EF36E010EDBCFF4FFF350F45CFE
:100FB0000BE2010EDB50EA6A520FE96E010EEA22E3
:100FC000EF6A010EDB2AEDD7030EDB6A040EDB6A43
:100FD000030EDBCF14F0040EDBCF15F0D8901550C4
:100FE00004E66C0E145C020E155839E28B928A905E
:100FF000030EE66EC0EC26F0E55282A424D0070E64
:10100000E76E030EDBCFF6FF040EDBCFF7FFE750F2
:10101000F616F76A8F0EF626470EF7220800F5CF70
:1010200014F0030EDBCFE9FF040EDBCFEAFF030E63
:10103000D890EA32E932E804FBE1520EE926010ECB
:10104000EA221450EF128B82030EE66EC0EC26F0FB
:10105000E552030EDB2A040EBBE3DB2AB9D78A82F2
:101060008B928A90030EE66EC0EC26F0E55282A4C5
:1010700008D0930EF66E470EF76E0800F55001018A
:101080009F138B820101800E006F020EE66EECEC66
:101090001AF0E552E66A7BEC1BF0E5528B92030EE8
:1010A000E66EC0EC26F0E5528A928B827F0E146EBB
:1010B0003B0E5FD2520E016F42C702F76DEC1BF080
:1010C000400E146E3B0E55D2520E016F42C702F70E
:1010D0006DEC1BF00101800E006F030EE66EECEC70
:1010E0001AF0E5528A920101526B01015C0E026F07
:1010F000020EDB6A080EF36E020EDBCFF4FFF35034
:10110000F45C49E28B92020EDB50070BF76A8F0FFB
:10111000F66E470EF7220800F5CF14F0020EDB4002
:10112000E840E8401F0BEA6A020FE96E010EEA226E
:10113000EF50141402E0010E01D0000E010BF36E0B
:10114000FE0E8A14F3108A6E030EE66EC0EC26F0D3
:10115000E55282A417D0020EDB50070BF76A8F0FFF
:10116000F66E470EF7220800F5CF14F0020EDB40B2
:10117000E840E8401F0BEA6A520FE96E010EEA22CE
:101180001450EF128B82030EE66EC0EC26F0E5528F
:10119000020EDB2AAFD70101529F5251E66EE66A7A
:1011A0001C0E146E3B0E156E166A14C0E6FFE66E3A
:1011B00016C0E6FFD950050FE66E000EDA20E66E87
:1011C0002BEC24F0F56E070EE15EF550D950050FBB
:1011D000E66E000EDA20E66E63EC13F0E552E5529F
:1011E0002E0E0101525D03E00701510E016F6DECFF
:1011F0001BF0CBD1520E016F42C702F7000E146EE6
:101200003B0E156E166A14C0E6FFE66E16C0E6FFCA
:1012100033EC13F0E552E552E552B3EC1BF0010E4E
:10122000DB6A500EF36E010EDBCFF4FFF350F45C7B
:1012300016E2010EDB50EA6A520FE96E010EEA2255
:10124000EF50E66E010EDB50EA6A020FE96E010E06
:10125000EA22E552E750EF6E010EDB2AE2D7030ED9
:10126000066E076A390EDBCF0BF03A0EDBCF0CF0BF
:10127000CEEC24F004C014F005C015F0010E1426C5
:10128000000E1522030E14C0DBFF040E15C0DBFF99
:10129000070EE76E030EDBCFF6FF040EDBCFF7FF82
:1012A000E750F616F76A8F0EF626470EF72208006B
:1012B000F5CF14F0030EDBCFE9FF040EDBCFEAFF1E
:1012C000030ED890EA32E932E804FBE1020EE92687
:1012D000010EEA221450EF123C0E0701415D24E09A
:1012E000070EE76E030EDBCFF6FF040EDBCFF7FF32
:1012F000E750F616F76A8F0EF626470EF72208001B
:10130000F51C146E030EDBCFE9FF040EDBCFEAFF02
:10131000030ED890EA32E932E804FBE1020EE92636
:10132000010EEA221450EF16030EDB2A040E01E32D
:10133000DB2A070EE76E030EDBCFF6FF040EDBCFD2
:10134000F7FFE750F616F76A8F0EF626470EF722DC
:101350000800F5CF14F0030EDBCFE9FF040EDBCF5E
:10136000EAFF030ED890EA32E932E804FBE1020E0C
:10137000E926010EEA221450EF123A0E0701415DF0
:1013800024E0070EE76E030EDBCFF6FF040EDBCF83
:10139000F7FFE750F616F76A8F0EF626470EF7228C
:1013A0000800F51C146E030EDBCFE9FF040EDBCF43
:1013B000EAFF030ED890EA32E932E804FBE1020EBC
:1013C000E926010EEA221450EF160101800E006F8B
:1013D000030EE66EECEC1AF0E5528A92010EDB6A1F
:1013E000500EF36E010EDBCFF4FFF350F45C0BE212
:1013F000010EDB50EA6A520FE96E010EEA22EF6A33
:10140000010EDB2AEDD7030EDB6A040EDB6A030E46
:10141000DBCF14F0040EDBCF15F0D890155004E6A6
:101420006C0E145C020E155866E28B92070EE76E86
:10143000030EDBCFF6FF040EDBCFF7FFE750F61607
:10144000F76A8F0EF626470EF7220800F5CF14F044
:10145000030EDBCFE9FF040EDBCFEAFF030ED890CB
:10146000EA32E932E804FBE1020EE926010EEA2243
:10147000EF50141402E0010E01D0000E010BF36EC8
:10148000FE0E8A14F3108A6E82A424D0070EE76E33
:10149000030EDBCFF6FF040EDBCFF7FFE750F616A7
:1014A000F76A8F0EF626470EF7220800F5CF14F0E4
:1014B000030EDBCFE9FF040EDBCFEAFF030ED8906B
:1014C000EA32E932E804FBE1520EE926010EEA2293
:1014D0001450EF12030EE66EC0EC26F0E5528B823C
:1014E000030EE66EC0EC26F0E552030EDB2A040E76
:1014F0008EE3DB2A8CD78A828B92930EF66E470E90
:10150000F76E0800F55001014F1502E0010E01D001
:10151000000E010BF36EFE0E8A14F3108A6E82A485
:1015200008D0930EF66E470EF76E0800F5500101D5
:101530009F138B820101800E006F020EE66EECECB1
:101540001AF0E552E66A7BEC1BF0E5528B92030E33
:10155000E66EC0EC26F0E5528A928B82E70E146E9E
:101560003A0E07D0510E016F080E026FD40E146EA2
:101570003A0E156E166A14C0E6FFE66E16C0E6FF58
:1015800033EC13F0E552E552E55204010CAF03D001
:101590003EEC22F0FAD73C0EE66E010EE66E070E28
:1015A000E66EA9EC21F0E552E552E552D9CFE1FF14
:1015B000E552E7CFD9FF1200D9CFE6FFE1CFD9FF3F
:1015C000710EE12604011351030A01E1F8D0010A6A
:1015D00001E0D1D1125101E0F2D0DF6A3C0EDF5CB4
:1015E00013E2DF50EA6A900FE96E040EEA22EF5030
:1015F000E66EDF50EA6AD00FE96E040EEA22E55289
:10160000E750EF6EDF2AEAD793C416F016C017F042
:10161000166A0401925100011610146E370E14C0A0
:10162000DBFF380E17C0DBFF370EDBCFE6FF380ECF
:10163000DBCFE6FF04019151E66EE66A9051E66E5B
:10164000E66AB40E146E3A0E156E166A14C0E6FF02
:10165000E66E16C0E6FFD950010FE66E000EDA20E6
:10166000E66E2BEC24F0F56E0B0EE15EF550D950D2
:10167000010FE66E000EDA20E66E63EC13F0E55221
:10168000E55204019051330A4DE0010A01E094D083
:101690000401530ED06F370EDBCF06F0380EDBCFD0
:1016A00007F0330E06C0DBFF340E07C0DBFF350E3C
:1016B000DB6A360EDB6A350EDBCF14F0360EDBCF7D
:1016C00015F004019151000115AE02D0D89003D05D
:1016D000145C000E155873E2330EDBCFE9FFDB2AF2
:1016E000340EDBCFEAFF01E3DB2A600EE926000EB1
:1016F000EA22EF50E66E350EDBCFE9FF360EDBCF88
:10170000EAFF040EE926000EEA22D00EE926040EB6
:10171000EA22E552E750EF6E350EDB2A360ECBE3B8
:10172000DB2AC9D70401500ED06F370EDBCF06F08D
:10173000380EDBCF07F0330E06C0DBFF340E07C0D8
:10174000DBFF350EDB6A360EDB6A350EDBCF14F0BD
:10175000360EDBCF15F004019151000115AE02D019
:10176000D89003D0145C000E155829E2350EDBCF5B
:10177000E9FF360EDBCFEAFF040EE926000EEA226F
:10178000900EE926040EEA22EF50E66E330EDBCF10
:10179000E9FFDB2A340EDBCFEAFF01E3DB2A600E30
:1017A000E926000EEA22E552E750EF6E350EDB2AFD
:1017B000360ECBE3DB2AC9D70401510ED06F0401EA
:1017C000125101E0D8D013C516F016C017F0166AF2
:1017D0000501125100011610146E6F0E14C0DBFFCC
:1017E000700E17C0DBFF6F0EDBCFE6FF700EDBCF96
:1017F000E6FF05011151E66EE66A1051E66EE66AF3
:10180000930E146E3A0E156E166A14C0E6FFE66E5D
:1018100016C0E6FFD950390FE66E000EDA20E66EEC
:101820002BEC24F0F56E0B0EE15EF550D950390F1C
:10183000E66E000EDA20E66E63EC13F0E552E55238
:1018400005011051330A4CE0010A01E092D0530E19
:10185000106F6F0EDBCF06F0700EDBCF07F06B0E54
:1018600006C0DBFF6C0E07C0DBFF6D0EDB6A6E0E81
:10187000DB6A6D0EDBCF14F06E0EDBCF15F00501C9
:101880001151000115AE02D0D89003D0145C000EA7
:10189000155871E26B0EDBCFE9FFDB2A6C0EDBCF54
:1018A000EAFF01E3DB2A600EE926000EEA22EF5090
:1018B000E66E6D0EDBCFE9FF6E0EDBCFEAFF040EA6
:1018C000E926000EEA22100EE926050EEA22E5526C
:1018D000E750EF6E6D0EDB2A6E0ECBE3DB2AC9D725
:1018E000500E106F6F0EDBCF06F0700EDBCF07F0DF
:1018F0006B0E06C0DBFF6C0E07C0DBFF6D0EDB6AF4
:101900006E0EDB6A6D0EDBCF14F06E0EDBCF15F0C2
:1019100005011151000115AE02D0D89003D0145C1E
:10192000000E155828E26D0EDBCFE9FF6E0EDBCFFF
:10193000EAFF040EE926000EEA22100EE926050E43
:10194000EA22EF50E66E6B0EDBCFE9FFDB2A6C0E6E
:10195000DBCFEAFF01E3DB2A600EE926000EEA2274
:10196000E552E750EF6E6D0EDB2A6E0ECBE3DB2AFD
:10197000C9D7510E106FD9CFE1FFE552E7CFD9FF9C
:1019800012000101AF51B01104E1280EAF6F230E18
:10199000B06FAF07000EB05B6DA208D0AF51B011B1
:1019A00030E18A7A8A50200B13E128D00001FB51E4
:1019B00002E18A9A23D0FB0502E18A8A09D0020E4D
:1019C000FB5D02E18A8A1AD0030EFB5D03E18A9A6D
:1019D0008A8C1200050EFB5D06E10101AF51B011CA
:1019E00010E18A7A0BD0060EFB5D0BE10101AF51CD
:1019F000B01107E18A7A8A50200B02E08A9C12001B
:101A00008A8C1200D9CFE6FFE6520101D00EA46FF6
:101A1000040EA56F01013C0EA86FE552E552E7CF19
:101A2000D9FF1200D9CFE6FFE6520101100EA46FD4
:101A3000050EA56F01013C0EA86FE552E552E7CFF8
:041A4000D9FF1200B8
:0C1A44005EEC12F0FB0EDBCFF3FFDB06C4
:101A5000F35000090AE0ACEC12F0FA0E17EC13F0A8
:101A6000F3E1151CF1E1010E01D0000E8DEF12F033
:101A70005EEC12F03B0EE12402E3E168E652E16E17
:101A8000010EDB6A020EDB6AF90EDBCFF6FFFA0EFF
:101A9000DBCFF7FFFB0EDBCFF8FF0800F550DF6E62
:101AA000DF5002E1B3EF11F0250EDF5C02E0A6EF9C
:101AB00011F0030EDB6A040EDB6A050EDB6A060E0C
:101AC000DB6A070EDB6AC6EC11F02D0EDF5C0CE062
:101AD0002B0EDF5C09E0200EDF5C06E0230EDF5CEE
:101AE00003E0300EDF5C1AE1DF50300A14E0130A25
:101AF0000FE0030A0AE00B0A05E0060AE4E1030E20
:101B0000DB80E1D7030EDB82DED7030EDB84DBD77D
:101B1000030EDB86D8D7030EDB88D5D72A0EDF5C11
:101B20001BE1C2EC11F010EC12F010E0030EDB80B0
:101B300006680768130EDBCF0BF0140EDBCF0CF03A
:101B4000ECEC24F0040E04C0DBFF03D0130EF9EC20
:101B500011F0C6EC11F00BD0090EDB6A67EC12F045
:101B600003E0DBEC12F0FAD7090EF9EC11F0030EEA
:101B7000DBB0DB982E0EDF5C1BE1C6EC11F02A0E09
:101B8000DF5C0BE1C2EC11F010EC12F003E1130E7C
:101B90004BEC12F0C6EC11F00BD0090EDB6A67ECCF
:101BA00012F003E0DBEC12F0FAD7090E4BEC12F066
:101BB000680EDF5C07E1C6EC11F0680EDF5C1DE12A
:101BC000030E18D0740EDF5C17E07A0EDF5C14E0B1
:101BD000480EDF5C06E0540EDF5C03E05A0EDF5C6B
:101BE00002E1020E07D06C0EDF5C03E06A0EDF5CE0
:101BF00004E1010E9EEC12F0C9DBDF506E0A01E138
:101C000081D31E0A01E192D1200A01E18FD13F0A5E
:101C100001E149D11A0A01E146D10D0A01E143D19E
:101C2000200A01E140D13A0A01E13DD1200A01E157
:101C30003AD1260A01E135D10D0A01E132D11A0A61
:101C400001E1D9D0200A4AE0300A1FE0460A0EE03E
:101C5000250A01E085D3D950F90FE96EFF0EDA208D
:101C6000EA6E010EEE5E000EEE5AEE5AACEC12F089
:101C7000250EE66E95DB03E1151C01E16BD3A8ECA4
:101C800012F001E26DD3DB2A6BD3080EDB6A040E7F
:101C9000DB50010806E2040EDB0470EC12F0DB50AE
:101CA0008BDB080EDB5009E0030EDB50010B05E176
:101CB00072DB01E04FD3080EDB6A64DBEFCFDFFF9E
:101CC00020EC13F003E1151C01E144D3A8EC12F061
:101CD00001E3DB2A60DB01E143D33CD3070EDB5099
:101CE00002080FE1ECEC12F0030EB3EC12F00E0E52
:101CF000EECFDBFF0F0EEECFDBFF100EEECFDBFFE4
:101D000020D0F70EDBCF17F0F80EDBCF18F0020E65
:101D1000175E000E185AF70E17C0DBFFF80E18C03A
:101D2000DBFF17C0E9FF18C0EAFFA3EC12F0166A48
:101D30000E0E14C0DBFF0F0E15C0DBFF100E16C019
:101D4000DBFF0E0EDBCFE6FF0F0EDBCFE6FF100E44
:101D5000DBCFE6FFD5EC25F0E552E552E552130E58
:101D600005C0DBFF140E06C0DBFF060EDB5005E0EE
:101D7000130EE7EC12F001E26ADB0BEC13F002E267
:101D8000130E37DBCEEC12F006E0040EE7EC12F097
:101D900002E2050E2EDB030EDBB005D0FCDA01E01B
:101DA000D9D2080EDB6A090EDB6A0E0EDBCFF6FF16
:101DB0000F0EDBCFF7FF100EDBCFF8FF0800F5505A
:101DC000DF6EDF5014E011EC13F011E220EC13F0A1
:101DD00003E1151C01E1BED2BBDB01E3DB2A090EE6
:101DE000DB2AD9500E0FE96E000ECBDBE7D7D3DA32
:101DF00001E1B6D2AFD2C6DA110EEECFDBFF120E82
:101E0000EDCFDBFF110EDBCFE6FF120EDBCFE6FFDF
:101E1000C7EC25F0E552E552130EF3CFDBFF140EAD
:101E2000F4CFDBFF060EDB5004E0130ED0DB01E243
:101E30000EDB0BEC13F002E2130EDBDAAFDB05E096
:101E4000040EC5DB02E2050ED4DA030EDBB005D0CA
:101E5000A2DA01E07FD2080EDB6A090EDB6A110EFE
:101E6000DBCFE9FF120EDBCFEAFFEFCFDFFFDF5062
:101E700014E0D7DB12E2E4DB03E1151C01E16AD2D6
:101E800067DB01E3DB2A090EDB2A110EDB2ADBCF3D
:101E9000E9FF120EE8E3DB2AE6D77DDA01E160D242
:101EA00059D2030EDB8E070EDB0410E195DB040E26
:101EB0005ADB0A0EEECFDBFF0B0EEECFDBFF0C0E74
:101EC000EECFDBFF0D0EEECFDBFF6CD0070EDB504D
:101ED00003082CE1030EDBAE0DD0B2DA020E76DA87
:101EE000EFCF14F0156A166A176A14AE39D0156868
:101EF000166835D0F70EDBCF15F0F80EDBCF16F0F5
:101F0000020E155E000E165AF70E15C0DBFFF80E16
:101F100016C0DBFF15C0E9FF16C0EAFFEFCF14F0D3
:101F20000A0E14C0DBFF0B0EDB6A38D0070EDB5045
:101F3000020809E1030EDBAE04D059DB16AE10D067
:101F40000ED055DB0DD0030EDBAE12D079DA020EC7
:101F50003DDAF9DA166A176A15AE02D01668176804
:101F6000E2DA0C0E16C0DBFF0D0E17C0DBFF1AD035
:101F7000F70EDBCF16F0F80EDBCF17F0020E165E71
:101F8000000E175AF70E16C0DBFFF80E17C0DBFF66
:101F900016C0E9FF17C0EAFFD6DAC5DA0C0EDB6A15
:101FA0000D0EDB6A060EDB5005E1010EF36E050E29
:101FB000F3CFDBFF150EDB6A160EDB6AD950370F45
:101FC000146E000EDA20156E390E14C0DBFF3A0EC7
:101FD00015C0DBFF380EDB6A080EDB6A0A0EAEDACC
:101FE000DF50780A12E0200A10E0280A0CE0200AEC
:101FF0000AE03F0A06E00D0A02E0200A08E1020EAC
:1020000005D0080E03D0080EDF26100E97DA030E57
:10201000DBBE02D0DB92DB94DB50800B26E08ADA59
:10202000030EEB50000AE8AE02D0D89008D0000EA4
:10203000EE5C000EEE58000EEE58000EEE5815E263
:1020400011DA09680A680B680C685BEC25F00A0E67
:1020500000C0DBFF0B0E01C0DBFF0C0E02C0DBFF7C
:102060000D0E03C0DBFF2D0E08D0030EDBA202D045
:102070002B0E03D0DBA408D0200EF36E170EF3CF87
:10208000DBFF150EDB2A02D0170EDB6A050EDB50D4
:1020900003E1B5D901E189D0960E146E4D0E156E8F
:1020A000000E166E070EDBCF17F0186A196A1A6A4F
:1020B00017C009F018C00AF019C00BF01AC00CF0D4
:1020C000D1D9FAEC25F014500024F36E15500120FC
:1020D000F46E16500220F86EF4CFF7FFF3CFF6FF40
:1020E0000800090EF5CFDBFF580EDF5C0FE1610E33
:1020F000F36E090E79D90AE3200E146E090EDBCFB8
:10210000E7FF1450E75E090EE7CFDBFF070EDBCFDA
:1021100014F0156A166A176A0DDA14C009F015C0B2
:102120000AF016C00BF017C00CF0EECF04F0EECFA3
:1021300005F0EECF06F0EFCF07F0FAEC25F007C080
:10214000EDFF06C0EDFF05C0EDFF04C0EFFF390E47
:10215000DBCFE9FFDB063A0EDBCFEAFF01E2DB066D
:10216000090EDBCFEFFF150EDB2A49D995E1030EEF
:10217000DBA61DD06F0EDF5C06E1BFD918E3150E9C
:10218000DB2859DA14D0780EDF5C09E0580EDF5CEA
:1021900006E0620EDF5C03E0420EDF5C08E1020E47
:1021A000F36E160EF3CFDBFF02D0150EDB6A030EC3
:1021B000DB50100B0EE0040EDBCF14F0050EDB50ED
:1021C000D880145406E2060EDB5003E1040EDB5007
:1021D00032DA93D90AE2050EDBCFE7FF150EDB50AA
:1021E000E75E050EE7CFDBFF02D0050EDB6A040ECB
:1021F000DBCF14F0160E43D9D880145414E2160E17
:10220000DBCFE6FF150EDBCFE6FF040EDBCFE6FFEC
:10221000050EDB50E552E75CE552D880E754E55205
:10222000D880E7545DD9030EDB50010B0BE1080E9B
:10223000DB5008E0B0D801E08DD0080EDB50BCD8F0
:10224000080EDB6A170EDB5007E086D9170EEFD9B0
:1022500003E1151C01E17ED0160EDB5016E07CD99F
:10226000300EE66E9DD802E1151C74E075D9DFCF03
:10227000E6FF19EC25F0E552E552E552F4CF15F0F2
:102280000001F31C02E1151C65E0050EDBCF14F024
:10229000160EDB50D880145409E2050EDBCFE7FFA1
:1022A000160EDB50E75E050EE7CFDBFF300EE66E65
:1022B000050EC9D94FE1390EDB2ADBCFE9FF3A0E13
:1022C00001E3DB2ADBCFEAFF090EEFCFDBFFDB50B8
:1022D0000EE042D9090EABD902E1151C3BE0390EE4
:1022E000DB2ADBCFE9FF3A0EEDE3DB2AEBD753D84D
:1022F00031E1160EDBCFE6FF080EC1D8E552E72428
:102300005BD82ED0070EDB50030A1CE0010A14E054
:10231000030A07E079D9DBCFEEFF020EDBCFEDFF3A
:102320001FD0F3D8196A17AE02D0186819682AD8D6
:10233000BAD819C0EEFF14D0E8D817BE186822D852
:10234000B2D80ED061D9DBCFEFFF0AD079D905E141
:10235000151C03E1F368F46810D0FAD801E3DB2A16
:1023600077D94DEF0DF0010EDBCF14F0020EDBCF6D
:1023700015F014C0F3FF15C0F4FFD9CFE1FFDACF99
:10238000E2FFCBD029D9020EB3EF12F061D90800D9
:10239000F550DF6E1200200EE66E080E23EF13F0EC
:1023A00019EC25F0E552E552E552F3CF14F0F4CFE5
:1023B00015F00001F31C1200146E156AD950010FBC
:1023C0004DD91450EE261550ED221200185E000E65
:1023D000195AF70E18C0DBFFF80E19C0DBFF18C042
:1023E000E9FF19C0EAFF1200DBCFF4FFF350F45C01
:1023F0001200DB50E76E040EE7CFDBFF12000A0E7F
:10240000DBCF14F00B0EDBCF15F00C0EDBCF16F08C
:102410000D0EDBCF17F01450151016101710120008
:10242000130EEECFDBFF140EEDCFDBFF130EDBCF71
:1024300014F0140EDBCF15F00001800E15141200FD
:10244000F70EDBCF18F0F80EDBCF19F01200050EF7
:10245000DB50E66ED950130F01D9E552E750EE6E0E
:10246000ED6A12000A0EDBCF04F00B0EDBCF05F095
:102470000C0EDBCF06F00D0EDBCF07F01200DBCF2A
:10248000E6FF150EDBCFE6FF050EDB50E552E72435
:10249000E552E7241200DB50CED8010EF36E060E93
:1024A000F3CFDBFF1200EE50EFCFEAFFE96E16C06C
:1024B000EEFF17C0EEFF18C0EEFF1200D9CFE6FF07
:1024C000DACFE6FFE1CFD9FFE2CFDAFF1200DFCFAC
:1024D000E6FFE66A83EC26F0E552E552F35012007F
:1024E000E76E080EE7CFDBFF1200EECF14F0EECF61
:1024F00015F0EFCF16F0176A1200050EDBCF14F0BF
:10250000150EDB50D88014541200010EDBCF16F0EC
:10251000020EDBCF17F0186A1200E552E5CFDAFFA2
:10252000E7CFD9FF12000A0E14C0DBFF0B0E15C057
:10253000DBFF1200D9500A0F2EEF13F0F36E070ED7
:10254000F3CFDBFF1200EECF14F0EFCF15F0120047
:10255000010EDB2A020E1200FC0EDBCFE6FFFD0EA1
:10256000DBCFE6FF1200145E000E155AF70E14C002
:10257000DBFFF80E15C0DBFF14C0E9FF15C0EAFF52
:102580001200DA20EA6EEF2AEECFF6FF000EEF22FD
:10259000EECFF7FFEF22EECFF8FF1200040EDBCFF5
:1025A000E6FF130EDB50E552E75C9ADFDB5004DFF9
:1025B000060EDB501200090EDB500A0DF350DF242B
:1025C000D00FE76E090EE7CFDBFFC6EF11F0DB504F
:1025D000F36E050EF4EF11F0F70EDBCF14F0F80EEA
:1025E000DBCF15F01200DFCFE6FFD0EF11F028DFD0
:1025F000030EECDE75EF12F022EC0DF0E552E55221
:10260000E552E55200091200BDDEEE50EFCFEAFFC1
:10261000E96E010E1200130EDB50F36E040EF4EFA0
:1026200011F0040EDB50F36E090EF4EF11F0DBCF66
:10263000E6FFD0EF11F0E76E050EE7CFDBFF1200EB
:102640008BDFF3EF12F0DBCFE6FF86DFFCEF12F05B
:10265000D950F90FE96EFF0EC1EF12F0E96E000ECE
:06266000DA20EA6E120010
:0A266600D9CFE6FFE1CFD9FFFC0E4B
:10267000DBCFF6FFFD0EDBCFF7FFFE0EDBCFF8FF63
:102680000800F5501CE0ACA2FED7FC0EDBCFF6FF35
:10269000FD0EDBCFF7FFFE0EDBCFF8FF0800F55095
:1026A000E66E6CEC26F0E552D950FC0FE96EFF0E99
:1026B000DA20EA6EEE2A000EEE22EE22D8D7E5529C
:1026C000E7CFD9FF1200D9CFE6FFE1CFD9FFFD0E4A
:1026D000DBCFE9FFFE0EDBCFEAFFEF5013E0ACA249
:1026E000FED7FD0EDBCFE9FFFE0EDBCFEAFFEF509A
:1026F000E66E6CEC26F0E552FD0EDB2AFE0EE7E3FB
:10270000DB2AE5D7E552E7CFD9FF1200D9CFE6FFA4
:10271000E1CFD9FF020EE126FC0EDB06DB50E76EAF
:10272000FD0EDBCFE9FFFE0EDBCFEAFFE750E92627
:10273000000EEA22EF6ADF6AFC0EDB50DF5C3EE24D
:102740009EAAFED71EEC26F0E76E010EE7CFDBFF58
:10275000FD0EDBCFE9FFFE0EDBCFEAFF010EDBCF84
:10276000EFFFACA2FED7010EDBCFE6FF6CEC26F04C
:10277000E552010EDB500D081AE1FD0EDBCFE9FF3B
:10278000DB2AFE0EDBCFEAFF01E3DB2A0A0EEF6E47
:10279000ACA2FED70A0EE66E6CEC26F0E552FD0EFA
:1027A000DBCFE9FFFE0EDBCFEAFFEF6A07D0FD0EBD
:1027B000DB2AFE0E01E3DB2ADF2ABED7D9CFE1FFF9
:1027C000E552E7CFD9FF1200D9CFE6FFE1CFD9FF1D
:1027D000660EE126070EDB6AF3EC17F08C6A6DECEF
:1027E0001BF0640E146E3A0E156E166A14C0E6FFE6
:1027F000E66E16C0E6FF37DFE552E552E5524A0EB7
:10280000146E3A0E156E166A14C0E6FFE66E16C018
:10281000E6FF29DFE552E552E5528CEC19F0DE6E59
:10282000DD6AD9CFE9FFDACFEAFFEE50ED100DE116
:102830003D0E146E3A0E156E166A14C0E6FFE66E73
:1028400016C0E6FF10DFE5522FD0DECFE6FFDDCF6A
:10285000E6FF360E146E3A0E156E166A14C0E6FFC9
:10286000E66E16C0E6FFD950090FE66E000EDA20BC
:10287000E66E2BEC24F0F56E070EE15EF5502E0EA1
:10288000146E3A0E156E166A14C0E6FFE66E16C098
:10289000E6FFE9DEE552E552E552D950090FE66E52
:1028A000000EDA20E66E0FDFE552E552020EE66E0C
:1028B00055EC26F0E552D950090F146EDACF15F019
:1028C000080EDB6A166A176A16BE176814501624BB
:1028D000E96E15501720EA6EEF6ABEDB9EAA69D238
:1028E0001EEC26F0E76E630EE7CFDBFFD950090F31
:1028F000146EDACF15F0080EDBCFF3FFDB2AF350AE
:10290000166E176A16BE176814501624E96E155015
:102910001720EA6E630EDBCFEFFFACA2FED7630E8B
:10292000DBCFE6FF6CEC26F0E552630EDB500D08C2
:1029300001E011D2D950090F146EDACF15F0080E4C
:10294000DB04166E176A16BE176814501624E96E5B
:1029500015501720EA6E0A0EEF6EACA2FED70A0ED3
:10296000E66E6CEC26F0E552D950090F146EDACF02
:1029700015F0080EDBCF16F0176A16BE1768145054
:102980001624E96E15501720EA6EEF6A280E146EB1
:102990003A0E156E166A14C0E6FFE66E16C0E6FF24
:1029A00062DEE552E552E552D950090FE66E000E9F
:1029B000DA20E66E88DEE552E552260EE66E3A0E25
:1029C000E66E81DEE552E552070EDB5012E0070E9F
:1029D000DB6A6DEC1BF0070E146E3A0E156E166A6C
:1029E00014C0E6FFE66E16C0E6FF3DDEE552E55296
:1029F000E552090EDB50610A01E1A0D1160A01E19E
:102A000054D1070A01E19AD1190A01E1BFD00D0A98
:102A100001E086D1F10E146E390E156E166A14C0DF
:102A2000E6FFE66E16C0E6FF1EDEE552E552E55211
:102A3000000EE66EE66A33EC18F0E552E552DE6A07
:102A4000DD6ADECF14F0DDCF15F0D890155004E626
:102A5000800E145C000E155801E370D1DECFE9FF43
:102A6000DDCFEAFF070EE926000EEA22600EE92616
:102A7000000EEA22EF50E66EE66ADECFE9FFDDCF18
:102A8000EAFF060EE926000EEA22600EE926000E95
:102A9000EA22EF50E66EE66ADECFE9FFDDCFEAFF1D
:102AA000050EE926000EEA22600EE926000EEA2253
:102AB000EF50E66EE66ADECFE9FFDDCFEAFF040EF7
:102AC000E926000EEA22600EE926000EEA22EF5007
:102AD000E66EE66ADECFE9FFDDCFEAFF030EE92608
:102AE000000EEA22600EE926000EEA22EF50E66EA2
:102AF000E66ADECFE9FFDDCFEAFF020EE926000E2F
:102B0000EA22600EE926000EEA22EF50E66EE66A3F
:102B1000DECFE9FFDDCFEAFF010EE926000EEA2253
:102B2000600EE926000EEA22EF50E66EE66ADECF7E
:102B3000E9FFDDCFEAFF600EE926000EEA22EF5042
:102B4000E66EE66AC50E146E390E156E166A14C06E
:102B5000E6FFE66E16C0E6FFD950090FE66E000EDE
:102B6000DA20E66E2BEC24F0F56E150EE15EF550E2
:102B7000D950090FE66E000EDA20E66EA4DDE552AC
:102B8000E552080EDE26000EDD225BD7D9500A0F73
:102B9000E66E000EDA20E66EE2EC22F0E552E55237
:102BA000020EF3CFDBFF030EF4CFDBFF020EDBCF11
:102BB00014F0030EDBCF15F0D890155004E6640E28
:102BC000145C000E15580DE3020EDBCF16F0030E59
:102BD000DBCF17F0173409E21650F408010E175432
:102BE00004E28F0E146E390E9ED0020EDBCFE6FF8C
:102BF000030EDBCFE6FF740E146E390E156E166AE7
:102C000014C0E6FFE66E16C0E6FFD950090FE66E67
:102C1000000EDA20E66E2BEC24F0F56E070EE15E76
:102C2000F550D950090FE66E000EDA20E66E4BDD46
:102C3000E552E552020EDE6EDD6ADECF14F0DDCF26
:102C400015F0D890155004E6800E145C000E15584F
:102C50000EE2DECFE9FFDDCFEAFF600EE926000ECF
:102C6000EA22EF6ADF2A010EE8E3DB2AE6D7FF0E4D
:102C7000E76E020EDBCF14F0030EDBCF15F0E7504A
:102C80001416156A14C060F0020EDBCF14F0030EA8
:102C9000DBCF15F015C014F0156A14C061F0000EFA
:102CA000E66EE66A94EC18F047D0390E146E390ED1
:102CB000156E166A14C0E6FFE66E16C0E6FFD3DC9A
:102CC000E552E552E552DE6ADD6ADECF14F0DDCF73
:102CD00015F0D890155004E6500E145C000E1558EF
:102CE0000EE2DECFE9FFDDCFEAFF020EE926010E9C
:102CF000EA22EF6ADF2A010EE8E3DB2AE6D74F0E6D
:102D0000F36E060EF3CFDBFF040EDB6A050EDB6A03
:102D10006DEC1BF0010EF36E070EF3CFDBFF0ED050
:102D20001B0E146E390E156E166A14C0E6FFE66EA1
:102D300016C0E6FF98DCE552E552E552D950090F7E
:102D4000146EDACF15F0080EDB6A166A176A16AE33
:102D500029D0176827D0080EDBCF14F0280EE76EB5
:102D60001418E8AE02D0143403D0E750D8801454BD
:102D700020E2FA0E146E380E156E166A14C0E6FFC5
:102D8000E66E16C0E6FF6FDCE552E552E552D9501B
:102D9000090F146EDACF15F0080EDB6A166A176A8F
:102DA00016BE176814501624E96E15501720EA6EE7
:102DB000EF6A26EC04F0070EDB5001E18ED54F0ED2
:102DC000F36E060EDBCFF4FFF350F45C03E2060E65
:102DD000DB2801D0000EE76E060EE7CFDBFFDB50ED
:102DE000F76A3F0FF66E470EF7220800F550F76AB4
:102DF000AE0FF66E460EF7220800F550030DF3CF26
:102E000014F0F4CF15F0020E1426000E1522020E57
:102E100014C0DBFF030E15C0DBFF070EE76E040EC8
:102E2000DBCFF6FF050EDBCFF7FFE750F616F76AAC
:102E30008F0EF626470EF7220800F51C146E040EBE
:102E4000DBCFE9FF050EDBCFEAFF030ED890EA32B5
:102E5000E932E804FBE1020EE926010EEA221450F1
:102E6000EF16070EE76E020EDBCFF6FF030EDBCF89
:102E7000F7FFE750F616F76A8F0EF626470EF72291
:102E80000800F5CF14F0020EDBCFE9FF030EDBCF15
:102E9000EAFFD890EA32E932E804FBE1020EE926C3
:102EA000010EEA221450EF12020EDBCF06F0030EE1
:102EB000DBCF07F0040E06C0DBFF050E07C0DBFF0B
:102EC000E66A7BEC1BF0E5520101400E006F040E38
:102ED000E66EECEC1AF0E5528A92640EDB6A650E3F
:102EE000DB6A640EDBCF14F0650EDBCF15F0D890F3
:102EF000155004E66C0E145C020E155845E28B92D8
:102F0000030EE66EC0EC26F0E552070EE76E640E87
:102F1000DBCFF6FF650EDBCFF7FFE750F616F76A5B
:102F20008F0EF626470EF7220800F5CF14F0640E38
:102F3000DBCFE9FF650EDBCFEAFF030ED890EA3264
:102F4000E932E804FBE1020EE926010EEA22EF5025
:102F5000141402E0010E01D0000E010BF36EFE0E00
:102F60008A14F3108A6E030EE66EC0EC26F0E5526A
:102F70008B82030EE66EC0EC26F0E552640EDB2A6F
:102F8000650EAFE3DB2AADD78A828B92930EF66E85
:102F9000470EF76E0800F55001014F1502E0010ED3
:102FA00001D0000E010BF36EFE0E8A14F3108A6E30
:102FB000030EE66EC0EC26F0E5528B820101800E16
:102FC000006F020EE66EECEC1AF0E552E66A7BEC5E
:102FD0001BF0E5528B92030EE66EC0EC26F0E55234
:102FE0008A928B827AD40F0EC11295689368899069
:102FF0008994180E926E8B8294928D8096908D8417
:1030000096948D829692899A929A8B8094909484C9
:10301000939093920101060EB16F9B0EE66EE66AE5
:103020003C0EE66E93EC25F0E552E552E552F40EC7
:10303000E66E95EC26F0E552140E6F6E0001FB6B08
:103040000001FC6B0001FD6B22EC04F09390939265
:103050000101060EB16F120022EC22F06FBE02D009
:063060003EEC22F012001C
:0A306600D9CFE6FFE1CFD9FF030E3A
:10307000E1260101050EB16F936A9568899AFE0EEB
:10308000DBCF15F015C014F0156A1450DF6EDF5059
:103090008A6E010EE66EC0EC26F0E552898AFF0EBC
:1030A000E76EFD0EDBCF14F0FE0EDBCF15F0E75020
:1030B0001416156A010E14C0DBFF8D848D90020E6C
:1030C000DB6ADB50146E156AD890155004E6800E4A
:1030D000145C000E155820E2020EDBCFE6FF010E55
:1030E000DB50E552E7108A6E8D92020EE66EC0EC60
:1030F00026F0E552020EDB50EA6A600FE96E000E20
:10310000EA2283CFEFFF8D82010EE66EC0EC26F03F
:10311000E552020EDB2AD5D78D809368D9CFE1FF27
:10312000E552E7CFD9FF1200D9CFE6FFE1CFD9FFB3
:10313000050EE1260101B16F936A956A8D82FE0E3C
:10314000DBCF15F015C014F0156A1450DF6E899AA4
:10315000DF508A6E020EE66EC0EC26F0E552898AD8
:10316000800EE76EFD0EDBCF14F0FE0EDBCF15F008
:10317000E7501416156A010E14C0DBFF8D90020E85
:10318000DB6ADB50146E156AD890155004E6800E89
:10319000145C000E155825E2020EDBCFE6FF010E8F
:1031A000DB50E552E7108A6E010EE66EC0EC26F0A9
:1031B000E5528D94020EDB50EA6A600FE96E000E54
:1031C000EA22EF508C6E010EE66EC0EC26F0E5525E
:1031D0008D84050EE66EC0EC26F0E552020EDB2A69
:1031E000D0D79568140EE66E55EC26F0E552800EA9
:1031F0000001DF15E76E020EE7CFDBFF200EF36E56
:10320000030EF3CFDBFF4E0EF36E040EF3CFDBFFA6
:10321000030EDBCF14F0040EDBCF15F015341EE2E5
:1032200014500008000E155419E28D92030EDB06AF
:10323000040E01E2DB06010EE66EC0EC26F0E5525C
:10324000800E8314146E020EDB50145C07E08D8236
:10325000010EE66EC0EC26F0E552DAD78D828D8045
:1032600093689568030EDBCF14F0040EDBCF15F0E6
:10327000153404E214500008000E155402E3010E48
:1032800001D0000ED9CFE1FFE552E7CFD9FF120000
:10329000D9CFE6FFE1CFD9FF020EE1260101050EED
:1032A000B16F936A9568899AFE0EDBCF15F015C051
:1032B00014F0156A1450DF6EDF508A6E020EE66E4F
:1032C000C0EC26F0E552898AFF0EE76EFD0EDBCFDB
:1032D00014F0FE0EDBCF15F0E7501416156A010E40
:1032E00014C0DBFF8D848D90DB508A6E020EE66E7B
:1032F000C0EC26F0E5528D92020EE66EC0EC26F090
:10330000E5528350DF6E8D828D80DF50D9CFE1FF93
:10331000E552E7CFD9FF1200D9CFE6FFE1CFD9FFC1
:103320002D0EE1260101070EB16F8A828A808B92F1
:10333000939293908990320EE66E55EC26F0E5520A
:1033400089808B90D00EDE6E070EDD6E030EDB6A79
:1033500080B610D0DF06010E01E2DB06D9CFE9FF0F
:10336000DACFEAFFEE50ED10F3E1020EF36E030E3A
:10337000F3CFDBFF8B80DE6ADD6ADECF14F0DDCFBA
:1033800015F0580E145C7F0E155801E3EFD0030EB4
:10339000DB5001E0EBD0DECF14F0DDCF15F0000EF6
:1033A0001426010E152214C0E6FF15C0E6FF5BDEF1
:1033B000E552E5528A828A808B9293929390020E14
:1033C000DB6ADB50146E156AD890155004E6800E47
:1033D000145C000E155801E3C0D08994020EDB5036
:1033E000EA6A600FE96E000EEA222C0EEFCFDBFFD7
:1033F000DB50010B02E0010E01D0000E010BF36E59
:10340000F346FD0E8914F310896E89848050100BE9
:1034100001E0A3D08050080B01E19FD089942C0ECD
:10342000DB50020B02E0010E01D0000E010BF36E27
:10343000F346FD0E8914F310896E89848050100BB9
:1034400001E08BD08050080B01E187D089942C0ECD
:10345000DB50040B02E0010E01D0000E010BF36EF5
:10346000F346FD0E8914F310896E89848050100B89
:1034700074E18050080B71E089942C0EDB50080B2E
:1034800002E0010E01D0000E010BF36EF346FD0EBB
:103490008914F310896E89848050100B5EE180508E
:1034A000080B5BE089942C0EDB50100B02E0010E40
:1034B00001D0000E010BF36EF346FD0E8914F310DC
:1034C000896E89848050100B48E18050080B45E0DC
:1034D00089942C0EDB50200B02E0010E01D0000E6F
:1034E000010BF36EF346FD0E8914F310896E898487
:1034F0008050100B32E18050080B2FE089942C0E85
:10350000DB50400B02E0010E01D0000E010BF36E08
:10351000F346FD0E8914F310896E89848050100BD8
:103520001CE18050080B19E089942C0EDB50800BB5
:1035300002E0010E01D0000E010BF36EF346FD0E0A
:103540008914F310896E89848050100B06E1805035
:10355000080B03E0020EDB2A34D780B807D080A620
:1035600005D0800EDE26000EDD2207D7DE6ADD6A7A
:10357000DECF14F0DDCF15F00A0E145C000E1558E6
:1035800011E28994010EE66EC0EC26F0E5528984C2
:10359000010EE66EC0EC26F0E552DF2A010EE8E3EC
:1035A000DB2AE6D78050080B02E08B8001D08B909D
:1035B000030EDB5009E18050080B080A01E0010E00
:1035C000E76E030EE7CFDBFF030EDB50D9CFE1FF41
:0835D000E552E7CFD9FF12001C
:0835D800D9CFE6FFE1CFD9FFD6
:1035E000FE0EDB50000815E28B92800E01010015E3
:1035F00002E0010E01D0000E010BF36EF346FD0E4A
:103600008A14F3108A6E009F00478B82FE0EDB0641
:10361000E7D7E552E7CFD9FF1200D9CFE6FFE1CFD8
:10362000D9FF040EE126030E02C1DBFFDE6ADD6A6C
:10363000080EF36E020EF3CFDBFFFD0EDBCF14F0AE
:10364000FE0EDBCF15F0153442E214500008000ED8
:1036500015543DE28B92030EDB50800B02E0010E0D
:1036600001D0000E010BF36EFE0E8A14F3108A6E69
:10367000030EDBCFF3FFF39EF346F3CFDBFF8B822A
:10368000020EDB06DBCF14F014341BE3D9CFE9FFC5
:10369000DACFEAFFEE2A000EED22EECFF3FFEDCFF8
:1036A000F4FFF3CFE9FFF4CFEAFF020EE926010EA3
:1036B000EA22030EEFCFDBFF080EF36E020EF3CF0C
:1036C000DBFFFD0EDB06FE0EB8E2DB06B6D7D9CF78
:1036D000E1FFE552E7CFD9FF12000101060EB16FFD
:1036E0009390948493920101F80E006F060EE66E9B
:1036F00073DFE5521200D9CFE6FFE1CFD9FFE652E2
:1037000002C1DFFF0101060EB16F93909484939282
:103710000101C00E006F040EE66E5EDFE552FE0E84
:10372000DBCF02F1020EE66EE66A77DFE552E55284
:103730000101C00E006FFE0EDB50200B02E0010EF7
:1037400001D0000E010BF36EFE0E8A14F3108A6E88
:10375000020EE66E41DFE552DFCF02F1E552E5529F
:10376000E7CFD9FF1200D9CFE6FFE1CFD9FF020E94
:10377000E126939293909484A00EE66EBCDFE5520E
:103780000101800E006F030EE66E26DFE5528A927D
:10379000DE6ADD6ADECF14F0DDCF15F0D89015506B
:1037A00004E6500E145C000E15580EE2DECFE9FF61
:1037B000DDCFEAFF520EE926010EEA22EF6ADF2A88
:1037C000010EE8E3DB2AE6D7DE6ADD6ADECF14F01D
:1037D000DDCF15F0D890155004E66C0E145C020E87
:1037E00015585BE28B92DECFF6FFDDCFF7FF070EB9
:1037F000F616000EF7168F0EF626470EF722080073
:10380000F5CF14F0DECFE9FFDDCFEAFF030ED8904D
:10381000EA32E932E804FBE1020EE926010EEA226F
:10382000EF50141402E0010E01D0000E010BF36EF4
:10383000FE0E8A14F3108A6E82A41FD0DECFF6FF2C
:10384000DDCFF7FF070EF616000EF7168F0EF626E1
:10385000470EF7220800F5CF14F0DECFE9FFDDCFE9
:10386000EAFF030ED890EA32E932E804FBE1520E97
:10387000E926010EEA221450EF12030EE66EC0ECA8
:1038800026F0E5528B82030EE66EC0EC26F0E55280
:10389000DF2A010E9BE3DB2A99D78A828B92930E53
:1038A000F66E470EF76E0800F55001014F1502E065
:1038B000010E01D0000E010BF36EFE0E8A14F31000
:1038C0008A6E82A407D0930EF66E470EF76E08003C
:1038D000F5509F138B82030EE66EC0EC26F0E55286
:1038E0000101800E006F020EE66E76DEE552D9CF42
:0A38F000E1FFE552E7CFD9FF120017
:0638FA002E2E2E206C6949
:103900006E6520746F6F206C6F6E672C2069676E18
:103910006F726564202E2E2E0D0A00636F6D6D612F
:103920006E64206E6F7420756E64657273746F6F51
:1039300064202E2E2E2E0D0A00626567696E207798
:10394000616C6B696E672D312773207061747465CB
:10395000726E202E2E2E207465726D696E617465F4
:1039600073206F6E206E65787420636F6D6D616E6D
:10397000640D0A003E3E20496E697469616C697A83
:10398000696E672063617264202325640D0A004319
:10399000617264206E756D626572206D757374203E
:1039A0006265206265747765656E20313030206114
:1039B0006E6420353030202E2E2E2069676E6F7297
:1039C00065640D0A002020253032782025303278B9
:1039D000202530327820253032782025303278206A
:1039E00025303278202530327820253032780D0A83
:1039F00000466972737420666C6173682073656336
:103A0000746F723A0D0A0077616C6B696E672D6F87
:103A10006E65732074657374207465726D696E6170
:103A20007465640D0A000D00436D643A2000666100
:103A3000696C65642000282564290D0A007375638C
:103A40006365737366756C0D0A002020465047410C
:103A500020636F6E66696775726174696F6E202E80
:103A60002E2E200045434520446967694C61622041
:103A700046504741206D6F6E69746F722028563131
:103A80002E30322920696E697469616C697A6564C7
:103A90000D0A005263766420466561747572652074
:103AA000727074202E2E2E2025642025642025304F
:103AB000780D0A0052637664204F75747075742017
:103AC000727074202E2E2E2025642025642025302F
:103AD000780D0A00556E6B6E6F776E206F702063E5
:103AE0006F6465210D0A0049523D455854455354B1
:103AF0002C206E6F7720696E2049444C450D0A00DA
:103B00004A54414720647269766520696E6469761B
:103B1000696475616C2070696E0D0A004A544147F2
:103B200020746573742E2073656E742035632C20A9
:103B3000726563656976656420253032780D0A0008
:103B40004A5441472072657365742E2049523D42A4
:103B500059504153532C206E6F7720696E20494491
:103B60004C450D0A004A544147206472697665202D
:103B7000616C6C2070696E73204C4F570D0A0049C0
:103B8000523D4558544553542C206E6F7720696E32
:103B90002049444C452073746174650D0A004A54F1
:103BA000414720647269766520616C6C2070696E93
:103BB0007320484947480D0A004A54414720636131
:103BC00070747572650D0A0020204552524F523AAA
:103BD000206D6179206E6F7420777269746520643E
:103BE000697265637420746F20666C61736820610C
:093BF0007420253034780D0A0020
:063BFA0004011051600BF4
:103C0000E842E842E842E842E842000901E01200E6
:103C10001151070A4CE00B0A4AE0070A3BE0010A8F
:103C200027E00B0A23E0020A21E0030A1DE0080A4C
:103C300012E0010A0EE00F0A0AE0030A01E0120096
:103C40000101010EA36F0001040EFB6F120058EF7B
:103C50001EF0AFEF1EF00101010EA36F0101FD0E7A
:103C6000A46F000EA56F10D0D6EF1EF021EF1FF04D
:103C70000101010EA36F040114510101A46FA56B92
:103C8000FE0EA427000EA5230001FC930101010EE6
:103C9000A86F12000101010EA36F04011451EA6A1A
:103CA000FE0FE96E000EEA2212C4EFFF12001200AE
:103CB000800E0401105D52E11351030A30E0010A45
:103CC0000CE0030A49E10101010EA36F0101970E07
:103CD000A46F470EA56F120E3CD00101010EA36F19
:103CE00004011251F66EF76AD890F636F736490E8F
:103CF000F626480EF7220900F5CFA4F10A00F5CF09
:103D0000A5F1020E0101F76AA425F66EA551F7226E
:103D10000900F5CFA8F10A00F5CFA9F11DD00101E6
:103D2000010EA36F04011251F66EF76AD890F636B1
:103D3000F7364D0EF626480EF7220900F5CFA4F10E
:103D40000A00F5CFA5F1A4C1F6FFA5C1F7FF080051
:103D5000F5500101A86FA96B0001FC83120001015D
:103D6000010EA36F0F0EE66E710EE66E0F0EE66E7D
:103D7000CDEC22F0E552E552E552010EE66EFE0E64
:103D8000E66E000EE66ECDEC22F0E552E552E5520D
:103D900012C4FDF00401125104E10001050EFB6F95
:103DA00012000001060EFB6F94EF21F00401506B2E
:103DB000516B040110511F0B020A13E0030A0DE0BE
:103DC000010A31E10101010EA36F040150810001DC
:103DD000FCA129D00401508326D00101010EA36F5C
:103DE00022D00101010EA36F040114510F0B080D25
:103DF000F350156A000F146E040E15221451800B37
:103E000001E0010E040DF35001011424A66F000E11
:103E10001520A76FA6C1E9FFEA6EEF50040B03E07F
:103E20000401010E506F0101A3050AE10101500ECA
:103E3000A46F040EA56F0001FC930101020EA86F90
:103E400012000401120510E110511F0B00090CE1D2
:103E50000101010EA36F030E0401115D03E10001D6
:103E6000FC8102D00001FC91040112513AE1105191
:103E70001F0B020836E114510F0B000932E001015B
:103E8000010EA36F040114510F0B080DF350156AB6
:103E9000000F146E040E15221451800B01E0010E68
:103EA000040DF35001011424A66F000E1520A76F16
:103EB000030E0401115D07E1840EA6C1E9FFA7C14D
:103EC000EAFFEF6E120014AF06D0A6C1E9FFA7C14A
:103ED000EAFFEF6A1200880EA6C1E9FFA7C1EAFF58
:043EE000EF6E12006F
:0C3EE4006C500BE1040100513C0BE84263
:103EF000E8420D0802E184EF1FF0B9EF1FF0040E55
:103F00006C5C01E14BD81200D9CFE6FFE1CFD9FFBD
:103F1000E6520101A26BA36BA86BA96BFDEC1DF02F
:103F2000DF6ADF50146E156A010E145C000E15581E
:103F30001AE20101A35117E1F76ADF34FE0BF736ED
:103F4000F66E530EF626480EF7220900F5CF14F050
:103F50000800F5CF15F004D015C0FAFF1450F96E23
:103F6000FBDFDF2ADED7D7D8E552E552E7CFD9FF0E
:103F70001200020E0101A25D0FE194D8020E0101B0
:103F8000A35D02E1DCEC0AF0040100BD02D0C80E22
:103F900001D0880E006F1200D0EF20F0040E000157
:103FA000FB5D09E112C46EFF6E50000802E2050ECF
:103FB00001D0030EFB6F0101A20509E10AD804013B
:103FC00004BD02D0C80E01D0880E046F1200D0EFDD
:103FD00020F0D9CFE6FFE1CFD9FF020EE1260101A3
:103FE000400EA85D000EA95905E2A8C1DEFFA9C1D7
:103FF000DDFF03D0400EDE6EDD6A04010493049100
:10400000010EDB500413DFCF05F4000EDB5001017D
:10401000A85F010EDB50A95B500EA66F040EA76FC0
:104020000001FCA31DD0D9CFE9FFDACFEAFFEE50A3
:10403000ED1032E0A4C1F6FFA5C1F7FF0800F5506E
:10404000A6C1E9FFA7C1EAFFEF6E0101A62B000E92
:10405000A723A42BA523DF06010EE5E2DB06E3D7A9
:10406000D9CFE9FFDACFEAFFEE50ED1015E0A4C199
:10407000E9FFA5C1EAFFEF50A6C1E9FFA7C1EAFF2A
:10408000EF6E0101A62B000EA723A42BA523DF06AC
:10409000010EE6E2DB06E4D7D9CFE1FFE552E7CF38
:1040A000D9FF1200D9CFE6FFE1CFD9FF020EE126FA
:1040B000030E04010015E76E010EE7CFDBFF01C41C
:1040C000DFFFDE500101A827DD50A923500EA46FA9
:1040D000040EA56FD9CFE9FFDACFEAFFEE50ED105D
:1040E00014E0A4C1E9FFA5C1EAFFEF50A6C1E9FFB2
:1040F000A7C1EAFFEF6EA62B000EA723A42BA523D2
:10410000DF06010EE7E2DB06E5D7D9CFE1FFE55296
:10411000E7CFD9FF12006D980101A3510BE1040113
:10412000400E016F100E026F040E036F840E006FBD
:10413000040123D0040110AF22D00101A8510401D1
:10414000165D0101A9510401175904E216C4A8F132
:1041500017C4A9F13EDF0101010EA26F0401400E58
:10416000016F100E026F040E036F800E006F0401CA
:10417000500E066F040E076FC80E046F1200010187
:10418000020EA26F0401056BC80E046F0401400EFD
:10419000016F500E026F040E036FC80E006F120005
:1041A0000101A26B0401400E016F100E026F040E9C
:0C41B000036F880E006F0401046B120006
:0441BC000401105199
:1041C0001F0B010801E01200145101E01200060E5D
:1041D000115D28E11351230A23E0010A0FE0030ACD
:1041E0001FE10101020EA36F0001FD0505E10101C0
:1041F000BB0EA46F470EA56F090E0FD00101020E72
:10420000A36F0001FD0505E101011A0EA46F480E20
:10421000A56F0001FD0504E12F0E0101A86FA96B38
:104220000001FC8304011051600BE842E842E842BF
:10423000E842E842010801E0120011510B0A2BE0AC
:10424000080A1BE0090A13E0080A09E00B0A05E066
:10425000080A01E0120051EF21F075EF21F0010191
:10426000020EA36F0101AA0EA46F010E0DD0010171
:10427000020EA36F13C4AAF112000101020EA36F74
:104280000101AB0EA46F010EA56F0001FC930101AB
:10429000010EA86F12000101020EA36F12C4ABF150
:1042A0001200D9CFE6FFE1CFD9FFE6520401135146
:1042B000030A0DE0020A12E11251010A0FE0010A9D
:1042C0000DE10101020EA36F02EC0DF007D01251B7
:1042D00005E10101020EA36F12EC0DF00001FC9349
:1042E000E552E552E7CFD9FF120004011351030A4A
:1042F0000FE0010A01E01200125101E01200010179
:10430000020EA36F0101900EA66F040EA76F12009C
:10431000125101E012000101020EA36F0101100E03
:10432000A66F050EA76F12000101AC6B1E0E716E19
:104330000401400E096F900E0A6F040E0B6F880E79
:10434000086F0401D00E0E6F040E0F6F400E0C6F3D
:104350001200D9CFE6FFE1CFD9FFE652FC0EDB50C9
:10436000400805E2400EF36EFC0EF3CFDBFFDF6A80
:10437000FC0EDB50DF5C19E2DF50E76EFD0EDBCF99
:10438000E9FFFE0EDBCFEAFFE750E926000EEA2246
:10439000EF50E66EDF50EA6AD00FE96E040EEA22B3
:1043A000E552E750EF6EDF2AE3D7FC0EDBCF0DF4CA
:1043B000400E04010C170C7D880E0C13E552E552DB
:1043C000E7CFD9FF1200D9CFE6FFE1CFD9FF010136
:1043D000AC6B040108BF30D0FC0EDBCF14F00951E8
:1043E000D880145403E2FC0E09C4DBFF0101AC6B5E
:1043F000FC0EDB50AC5D19E2AC51EA6A900FE96E3D
:10440000040EEA22EF50E66EAC51E76EFD0EDBCFF4
:10441000E9FFFE0EDBCFEAFFE750E926000EEA22B5
:10442000E552E750EF6EAC2BE3D70401400E096F65
:104430000817087D880E08130101AC51E552E7CF3B
:04444000D9FF12008E
:0C4444006DA60CD80001FB0508E16DBA64
:1044500006D0686A696A69806988020EFB6F12007B
:104460006D6A696A6D860001010EFB6F12006D6A4C
:10447000696A0001FB6B120037EF22F00001FB516B
:1044800001E112006850040B04E06950040B01E0E4
:1044900041D86DB212006850010B04E06950010B65
:1044A00001E059D86850100B04E06950100B01E08E
:1044B00024D86850400B04E06950400B01E040D81C
:1044C0006850200B04E06950200B01E03BD8685095
:1044D000020B04E06950020B01E03BD8030E00011F
:1044E000FB5D01E212006850080B06E06950080B02
:1044F00003E072EC1FF068961200698468986D8280
:10450000A19AF290A08AF2860300F2B007D8A09A8E
:10451000F29612006D926994689412000001FCA159
:104520000ED0F8DF6D840101080EAD6F070EAE6F7F
:10453000AD07000EAE5BAD51AE11FAE16D94120005
:10454000689C120070A003D0D0EC20F07090689AA4
:104550001200689212006A6A686A9F0E6B6E7B0E88
:10456000696E6E6A0F0EE66E710EE66E0F0EE66EE7
:1045700014D8E552E552E552160E706E68A602D0C8
:104580006896FCD76D98D0EC20F00001FC910001FA
:10459000FD6B0001030EFB6F1200D9CFE6FFE1CFE8
:1045A000D9FFFD0EDBCFE9FFFE0EDBCFEAFFFC0EED
:1045B000DB5004E0EE6AFC0EDB06F9D7E552E7CFEC
:0445C000D9FF12000D
:0C45C400FF0EE3CFEAFFE552FF0EE3CF4D
:1045D000E9FFE552E66AE66AD9CFE6FFDACFE6FF01
:1045E000FC0EE124D96EFF0EE220DA6EE66AE66A7E
:1045F000E66A200EEF5C06E0090EEF5C03E0EF6672
:1046000003D03FD0EE50F5D72D0EEF5C03E1FF0E47
:10461000E32A03D02B0EEF5C01E1EE502F0EEF6486
:1046200024D03A0EEF6021D0D890F90EE336FA0E7E
:10463000E336FD0EDECFE3FFFE0EDDCFE3FFD890C5
:10464000F90EE336FA0EE336D890F90EE336FA0E99
:10465000E336FD0EE350DE26FE0EE350DD22300E83
:10466000EE5CDE26000EDD22D9D7FF0EE3CFE8FF99
:10467000E85207E0F90EE31EE32AFA0ED8B4E30687
:10468000E31EE552E552E552FF0EE3CFDAFFE552B5
:10469000FF0EE3CFD9FFE552E1CFE9FFE2CFEAFF1A
:0E46A000ED52ED52EECFF3FFEFCFF4FF12001C
:0246AE000011F9
:1046B000100C00000000080705040100CECDCBC996
:1046C0000000C9C7C5C3C1BFBD00BBB9000000B869
:1046D00000B3B1AFAEADACABAAA8A6A4A29F9E9CFE
:1046E0009A999800000000949391908E8C89878607
:1046F0008381807F7E7D7C00757400000072706E07
:104700006D6B6A6968666463000062615F5D5B5936
:104710005857545300000000504F4C4746454443FF
:10472000413F3D3C3B3937353432302E00002D2B94
:104730002927262423211F1D1B19181716151417A6
:104740001615100F0E0C0B0A0908030201908F8E2C
:104750008D8C8B8A898887868584837A796D6C6B4A
:104760006A65636260115C18191A1C1D23242526D2
:104770002728292A2B2C2D2E2F3031323334393A49
:104780003B3C3D3E3F4041424344454748145980ED
:0747900040201008040201A3
:094797001201000200000040259F
:1047A000099912010001020001090229000101001A
:1047B000A0320904000002030000000921010100E9
:1047C00001222F000705810340000A07050103406D
:1047D000000A040309041E0355004300530042006D
:1047E0002F00450043004500200044006500700094
:1047F00074002E00260344006900670069004C0025
:104800006100620020004600500047004100200087
:1048100062006F0061007200640006A0FF0901A140
:1048200001090315002600FF7508953C8102090463
:1048300015002600FF7508953C9102090515002614
:1048400000FF7508953CB102C0A947A947D247D6D9
:0548500047F447BC41E4
:0A485600D9CFE6FFDACFE6FFE1CF8D
:10486000D9FFE2CFDAFFE652E652E652E652D950DD
:10487000F90F146EFF0EDA20156E020E14C0DBFF66
:10488000030E15C0DBFF020EDBCFE6FF030EDBCF0E
:10489000E6FFF90EDBCFE6FFFA0EDBCFE6FFFB0EFD
:1048A000DBCFE6FFD950FC0FE66EFF0EDA20E66E96
:1048B00038EC0DF0F56E070EE15C02E2E16AE552BC
:1048C000E16EF550F3CFDEFFF4CFDDFFFC0EDBCF62
:1048D000E9FFFD0EDBCFEAFFEF6ADECF14F0DDCF9C
:1048E00015F014C0F3FF15C0F4FFD9CFE1FFDACF04
:0E48F000E2FFE552E5CFDAFFE7CFD9FF120075
:0248FE002A0E80
:10490000F66E080EF76E000EF86E00010900F55005
:10491000F66F0900F550F76F03E1F66701D03DD05F
:104920000900F550F16F0900F550F26F0900F550DC
:10493000F36F09000900F550E96E0900F550EA6EC1
:10494000090009000900F550F46F0900F550F56FF2
:1049500009000900F6CFF8F0F7CFF9F0F8CFFAF038
:10496000F1C0F6FFF2C0F7FFF3C0F8FF0001F45307
:1049700002E1F55307E00900F550EE6EF407F8E2A6
:10498000F507F9D7F8C0F6FFF9C0F7FFFAC0F8FF4E
:0C4990000001F607000EF75BBFD7120015
:04499C0006C012F04F
:1049A00006500B02F4CF05F0F3CF04F007500C02D1
:1049B000F4CF07F0F3CF06F00B02F3500526F450C6
:1049C0000622E86A072212500C02F3500526F45022
:1049D0000622E86A0722000C07C013F006C012F096
:1049E00006500B02F4CF05F0F3CF04F007500C0291
:1049F000F4CF07F0F3CF06F00B02F3500526F45086
:104A00000622E86A072212500C02F3500526F450E1
:104A10000622E86A07220CAE12EF25F01250065E5D
:104A20001350075A13AE000C0B50065E0C50075A79
:024A3000000C78
:0E4A3200D9CFE6FFDACFE6FFE1CFD9FFE2CF22
:104A4000DAFFFB0EDBCF14F0FC0EDBCF15F000011C
:104A5000800E15141AE1FB0EDBCFE9FFFC0EDBCF55
:104A6000EAFFEECFF3FFEDCFF4FFEE2A000EEF22C8
:104A7000F3CFE9FFF4CFEAFFFD0EDBCFEFFFEF50FE
:104A8000156AF36E15C0F4FF10D0FB0EDB50FE0864
:104A900006E1FD0EDBCFE6FFA6EC26F005D0FD0E0D
:104AA000DBCFE6FFD4EC26F0E552E552E5CFDAFFA6
:064AB000E7CFD9FF120060
:0A4AB60004500902F3CF00F0F4CF22
:104AC00001F00A02F3500126000EF420026E045099
:104AD0000B02F3500226000EF420036E04500C0269
:104AE000F350032605500902F3500126F450022228
:104AF000000E032205500A02F3500226F45003224E
:104B000005500B02F350032606500902F35002260B
:104B1000F450032206500A02F350032607500902FC
:064B2000F3500326120011
:0A4B2600D9CFE6FFDACFE6FFE1CFBA
:104B3000D9FFE2CFDAFFAC6AAB6AFD0EDBB0AC881E
:104B4000DBA202D0AC8CAB8CDBB4AC8EDBA602D08B
:104B5000AB8801D0AB8ADBA802D0AC8401D0AC9486
:104B60009E98DBAC02D09D8A01D09D9A9E9ADBAEC6
:104B700002D09D8801D09D98FB0EDB50AF6EAC8AB1
:0E4B8000AB8EE552E5CFDAFFE7CFD9FF12008A
:024B8E00FE0E19
:104B9000E3CFE9FFFF0EE3CFEAFFF36AF46AEE52D8
:104BA00003E0F34AF42AFBD71200FF0EE3CFF8FF2D
:104BB000E552FF0EE3CFF7FFE552FF0EE3CFF6FF1E
:104BC000E552E66AE66AE66A0900F55209E0FD0E7A
:104BD000E32A05E1FE0EE32A02E1FF0EE32AF4D701
:104BE000FD0EE3CF05F0FE0EE3CF06F0FF0EE3CFA0
:044BF00007F01200B8
:0C4BF400036A026A016A006A200EE76E84
:104C0000D8900436053606360736003601360236A9
:104C100003360950005C0A5001580B5002580C50E2
:104C2000035809E30950005E0A50015A0B50025A1A
:0C4C30000C50035A042AE72EE4D71200AF
:044C3C00D9CFE6FFE7
:104C4000DACFE6FFE1CFD9FFE2CFDAFFE652F00E8E
:104C50000001FF17ABAC03D0FF91ABB0FF81ABB449
:104C6000FF85ABB2FF87AE50DF6EDF50E552E552F5
:0A4C7000E5CFDAFFE7CFD9FF12000D
:064C7A00DACFE4FFE65270
:104C8000E552E5CFDAFF1100D8CFE4FFE0CFE4FF33
:104C9000E46EDACFE4FFE652E552E5CFDAFFE55005
:0A4CA000E5CFE0FFE5CFD8FF1000DC
:064CAA00FF0EE3501C6E3A
:104CB000EF0E01D0F30EE76EE72E5CEF26F00C0E40
:104CC0001B6EE76AE72E62EF26F01B2E61EF26F0DF
:084CD0001C2E5AEF26F0120021
:084CD800D9CFE6FFDACFE6FFB9
:104CE000E1CFD9FFE2CFDAFFACAC04D0AC90000149
:104CF000FFB3AC80FD0EDB50AD6EE552E5CFDAFFC1
:064D0000E7CFD9FF12000D
:0A4D0600F36AF46AFF0EE124E96E7F
:104D1000FF0EE220EA6EED6607D02F0EEF6404D09E
:0A4D20003A0EEF6001D0F32A1200F2
:064D2A00D9CFE6FFDACF4D
:104D3000E6FFE1CFD9FFE2CFDAFFFD0EDB50B86E20
:0C4D4000E552E5CFDAFFE7CFD9FF120003
:044D4C00FF0EE35023
:104D5000ACBA04D0AF6AAB8EAC8A949CACA2FED73E
:084D6000AD6EF36EF46A12005F
:084D680013EE00F023EE00F051
:104D7000F86A0F9C7FEC24F0E4EC13F0FDD71200EE
:104D8000FF0EE350E84E1200000000D000D000D02B
:064D9000E82EFAD7120024
:0A4D96003031323334353637383906
:074DA00061626364656600B7
:024DA8001200F7
:024DAA00000007
:044DAC00303132333D
:0D4DB000343536373839616263646566005A
:020000040030CA
:0100000024DB
:010001000EF0
:010002003FBE
:010003001EDE
:010005008179
:010006008178
:010008000FE8
:01000900C036
:01000A000FE6
:01000B00A054
:01000C000FE4
:01000D0040B2
:00000001FF
